 objsize001

 Timestamp is 31f090ea (reproducible build file hash)

 Preferred load address is 0000000180000000

 Start         Length     Name                   Class
 0001:00000000 00003950H .text$mn                CODE
 0001:00003950 00000036H .text$mn$00             CODE
 0001:00003986 00000092H .text$x                 CODE
 0002:00000000 000001c8H .idata$5                DATA
 0002:000001c8 00000038H .00cfg                  DATA
 0002:00000200 00000008H .CRT$XCA                DATA
 0002:00000208 00000008H .CRT$XCZ                DATA
 0002:00000210 00000008H .CRT$XIA                DATA
 0002:00000218 00000008H .CRT$XIC                DATA
 0002:00000220 00000008H .CRT$XIZ                DATA
 0002:00000228 00000008H .CRT$XLA                DATA
 0002:00000230 00000008H .CRT$XLZ                DATA
 0002:00000238 00000008H .CRT$XPA                DATA
 0002:00000240 00000008H .CRT$XPZ                DATA
 0002:00000248 00000008H .CRT$XTA                DATA
 0002:00000250 00000010H .CRT$XTZ                DATA
 0002:00000258 00000000H .gehcont$y              DATA
 0002:00000258 00000000H .gfids$y                DATA
 0002:00000260 000024a0H .rdata                  DATA
 0002:00002700 00000000H .rdata$CastGuardVftablesA DATA
 0002:00002700 00000000H .rdata$CastGuardVftablesC DATA
 0002:00002700 00000028H .rdata$T                DATA
 0002:00002728 000000bcH .rdata$voltmd           DATA
 0002:000027e4 0000031cH .rdata$zzzdbg           DATA
 0002:00002b00 00000008H .rtc$IAA                DATA
 0002:00002b08 00000008H .rtc$IZZ                DATA
 0002:00002b10 00000008H .rtc$TAA                DATA
 0002:00002b18 00000008H .rtc$TZZ                DATA
 0002:00002b20 00000004H .tls                    DATA
 0002:00002b24 00000004H .tls$                   DATA
 0002:00002b28 00000008H .tls$ZZZ                DATA
 0002:00002b30 00000340H .xdata                  DATA
 0002:00002e70 00000364H .edata                  DATA
 0002:000031d4 0000008cH .idata$2                DATA
 0002:00003260 00000018H .idata$3                DATA
 0002:00003278 000001c8H .idata$4                DATA
 0002:00003440 00000486H .idata$6                DATA
 0003:00000000 00000080H .data                   DATA
 0003:00000080 0001b238H .bss                    DATA
 0004:00000000 000003c0H .pdata                  DATA

  Address         Publics by Value              Rva+Base               Lib:Object

 0000:00000000       __AbsoluteZero             0000000000000000     <absolute>
 0000:00000000       ___safe_se_handler_count   0000000000000000     <absolute>
 0000:00000000       ___safe_se_handler_table   0000000000000000     <absolute>
 0000:00000000       __arm64x_extra_rfe_table   0000000000000000     <absolute>
 0000:00000000       __arm64x_extra_rfe_table_size 0000000000000000     <absolute>
 0000:00000000       __arm64x_native_entrypoint 0000000000000000     <absolute>
 0000:00000000       __arm64x_redirection_metadata 0000000000000000     <absolute>
 0000:00000000       __arm64x_redirection_metadata_count 0000000000000000     <absolute>
 0000:00000000       __dynamic_value_reloc_table 0000000000000000     <absolute>
 0000:00000000       __enclave_config           0000000000000000     <absolute>
 0000:00000000       __guard_check_icall_a64n_fptr 0000000000000000     <absolute>
 0000:00000000       __guard_eh_cont_count      0000000000000000     <absolute>
 0000:00000000       __guard_eh_cont_table      0000000000000000     <absolute>
 0000:00000000       __guard_fids_count         0000000000000000     <absolute>
 0000:00000000       __guard_fids_table         0000000000000000     <absolute>
 0000:00000000       __guard_iat_count          0000000000000000     <absolute>
 0000:00000000       __guard_iat_table          0000000000000000     <absolute>
 0000:00000000       __guard_longjmp_count      0000000000000000     <absolute>
 0000:00000000       __guard_longjmp_table      0000000000000000     <absolute>
 0000:00000000       __hybrid_auxiliary_iat     0000000000000000     <absolute>
 0000:00000000       __hybrid_auxiliary_iat_copy 0000000000000000     <absolute>
 0000:00000000       __hybrid_code_map          0000000000000000     <absolute>
 0000:00000000       __hybrid_code_map_count    0000000000000000     <absolute>
 0000:00000000       __x64_code_ranges_to_entry_points 0000000000000000     <absolute>
 0000:00000000       __x64_code_ranges_to_entry_points_count 0000000000000000     <absolute>
 0000:00000100       __guard_flags              0000000000000100     <absolute>
 0000:00000000       __ImageBase                0000000180000000     <linker-defined>
 0001:00000000       ?NewObject@JNIEnv_@@QEAAPEAV_jobject@@PEAV_jclass@@PEAU_jmethodID@@ZZ 0000000180001000 f i libobjsize001.obj
 0001:00000028       ?TranslateError@@YAPEBDW4jvmtiError@@@Z 0000000180001028 f   libobjsize001.obj
 0001:000002e0       ?nsk_jni_check_exception@@YAHPEAUJNIEnv_@@QEBDH@Z 00000001800012e0 f   libobjsize001.obj
 0001:00000424       ?nsk_jni_lverify@@YAHHPEAUJNIEnv_@@HQEBDH1ZZ 0000000180001424 f   libobjsize001.obj
 0001:000004c4       Agent_Initialize           00000001800014c4 f   libobjsize001.obj
 0001:00000628       Agent_OnAttach             0000000180001628 f   libobjsize001.obj
 0001:00000628       Agent_OnLoad               0000000180001628 f   libobjsize001.obj
 0001:00000630       Java_nsk_jvmti_unit_FollowReferences_FollowRefObjects_addRefToVerify 0000000180001630 f   libobjsize001.obj
 0001:00000808       Java_nsk_jvmti_unit_FollowReferences_FollowRefObjects_getTag 0000000180001808 f   libobjsize001.obj
 0001:000008c8       Java_nsk_jvmti_unit_FollowReferences_FollowRefObjects_resetRefsToVerify 00000001800018c8 f   libobjsize001.obj
 0001:000008d0       Java_nsk_jvmti_unit_FollowReferences_FollowRefObjects_resetTags 00000001800018d0 f   libobjsize001.obj
 0001:00000914       Java_nsk_jvmti_unit_FollowReferences_FollowRefObjects_setTag 0000000180001914 f   libobjsize001.obj
 0001:00000b6c       Java_nsk_share_jvmti_ArgumentHandler_getAgentOptionsString 0000000180001b6c f   libobjsize001.obj
 0001:00000c1c       Java_nsk_share_jvmti_DebugeeClass_checkStatus 0000000180001c1c f   libobjsize001.obj
 0001:00000ca4       Java_nsk_share_jvmti_DebugeeClass_resetAgentData 0000000180001ca4 f   libobjsize001.obj
 0001:00000d04       Java_nsk_share_jvmti_RedefineAgent_agentStatus 0000000180001d04 f   libobjsize001.obj
 0001:00000d10       Java_nsk_share_jvmti_RedefineAgent_isRedefined 0000000180001d10 f   libobjsize001.obj
 0001:00000d1c       Java_nsk_share_jvmti_RedefineAgent_redefineAttempted 0000000180001d1c f   libobjsize001.obj
 0001:00000d28       MA_checkStatus             0000000180001d28 f   libobjsize001.obj
 0001:00000dcc       __local_stdio_printf_options 0000000180001dcc f i libobjsize001.obj
 0001:00001908       exitOnError                0000000180002908 f   libobjsize001.obj
 0001:000019bc       fprintf                    00000001800029bc f i libobjsize001.obj
 0001:00001a00       nsk_complain               0000000180002a00 f   libobjsize001.obj
 0001:00001a2c       nsk_jvmti_createJVMTIEnv   0000000180002a2c f   libobjsize001.obj
 0001:00001b5c       nsk_jvmti_lverify          0000000180002b5c f   libobjsize001.obj
 0001:00001c4c       nsk_jvmti_parseOptions     0000000180002c4c f   libobjsize001.obj
 0001:00001e9c       nsk_jvmti_resetAgentData   0000000180002e9c f   libobjsize001.obj
 0001:00001f1c       nsk_jvmti_resumeSync       0000000180002f1c f   libobjsize001.obj
 0001:00001fc4       nsk_jvmti_setFailStatus    0000000180002fc4 f   libobjsize001.obj
 0001:00002000       nsk_jvmti_waitForSync      0000000180003000 f   libobjsize001.obj
 0001:00002104       nsk_lcomplain              0000000180003104 f   libobjsize001.obj
 0001:00002124       nsk_ldisplay               0000000180003124 f   libobjsize001.obj
 0001:00002144       nsk_ltrace                 0000000180003144 f   libobjsize001.obj
 0001:00002164       nsk_lvcomplain             0000000180003164 f   libobjsize001.obj
 0001:0000231c       nsk_lvdisplay              000000018000331c f   libobjsize001.obj
 0001:00002368       nsk_lverify                0000000180003368 f   libobjsize001.obj
 0001:000023c4       nsk_lvtrace                00000001800033c4 f   libobjsize001.obj
 0001:00002424       nsk_printf                 0000000180003424 f   libobjsize001.obj
 0001:0000244c       nsk_vprintf                000000018000344c f   libobjsize001.obj
 0001:00002500       printf                     0000000180003500 f i libobjsize001.obj
 0001:00002a28       __raise_securityfailure    0000000180003a28 f   MSVCRT:gs_report.obj
 0001:00002a5c       __report_gsfailure         0000000180003a5c f   MSVCRT:gs_report.obj
 0001:00002c9c       __GSHandlerCheck           0000000180003c9c f   MSVCRT:gshandler.obj
 0001:00002cbc       __GSHandlerCheckCommon     0000000180003cbc f   MSVCRT:gshandler.obj
 0001:00002d30       __security_check_cookie    0000000180003d30 f   MSVCRT:amdsecgs.obj
 0001:00003070       _DllMainCRTStartup         0000000180004070 f   MSVCRT:dll_dllmain.obj
 0001:000030b0       __scrt_acquire_startup_lock 00000001800040b0 f   MSVCRT:utility.obj
 0001:000030ec       __scrt_dllmain_after_initialize_c 00000001800040ec f   MSVCRT:utility.obj
 0001:00003120       __scrt_dllmain_before_initialize_c 0000000180004120 f   MSVCRT:utility.obj
 0001:00003138       __scrt_dllmain_crt_thread_attach 0000000180004138 f   MSVCRT:utility.obj
 0001:00003160       __scrt_dllmain_crt_thread_detach 0000000180004160 f   MSVCRT:utility.obj
 0001:00003178       __scrt_dllmain_exception_filter 0000000180004178 f   MSVCRT:utility.obj
 0001:000031d8       __scrt_dllmain_uninitialize_c 00000001800041d8 f   MSVCRT:utility.obj
 0001:00003208       __scrt_dllmain_uninitialize_critical 0000000180004208 f   MSVCRT:utility.obj
 0001:0000321c       __scrt_initialize_crt      000000018000421c f   MSVCRT:utility.obj
 0001:00003268       __scrt_initialize_onexit_tables 0000000180004268 f   MSVCRT:utility.obj
 0001:000032f4       __scrt_is_nonwritable_in_current_image 00000001800042f4 f   MSVCRT:utility.obj
 0001:0000338c       __scrt_release_startup_lock 000000018000438c f   MSVCRT:utility.obj
 0001:000033b0       __scrt_uninitialize_crt    00000001800043b0 f   MSVCRT:utility.obj
 0001:000033dc       _onexit                    00000001800043dc f   MSVCRT:utility.obj
 0001:00003418       atexit                     0000000180004418 f   MSVCRT:utility.obj
 0001:00003430       __crt_debugger_hook        0000000180004430 f   MSVCRT:utility_desktop.obj
 0001:00003438       __scrt_fastfail            0000000180004438 f   MSVCRT:utility_desktop.obj
 0001:00003584       _guard_check_icall_nop     0000000180004584 f i MSVCRT:guard_support.obj
 0001:00003588       __security_init_cookie     0000000180004588 f   MSVCRT:gs_support.obj
 0001:00003634       DllMain                    0000000180004634 f   MSVCRT:dll_dllmain_stub.obj
 0001:00003658       ?__scrt_initialize_type_info@@YAXXZ 0000000180004658 f   MSVCRT:tncleanup.obj
 0001:00003668       ?__scrt_uninitialize_type_info@@YAXXZ 0000000180004668 f   MSVCRT:tncleanup.obj
 0001:00003674       __local_stdio_scanf_options 0000000180004674 f i MSVCRT:default_local_stdio_options.obj
 0001:0000367c       __scrt_initialize_default_local_stdio_options 000000018000467c f   MSVCRT:default_local_stdio_options.obj
 0001:00003698       __scrt_get_dyn_tls_init_callback 0000000180004698 f   MSVCRT:dyn_tls_init.obj
 0001:000036a0       _RTC_Initialize            00000001800046a0 f   MSVCRT:initsect.obj
 0001:000036dc       _RTC_Terminate             00000001800046dc f   MSVCRT:initsect.obj
 0001:00003718       __isa_available_init       0000000180004718 f   MSVCRT:cpu_disp.obj
 0001:000038c4       _get_startup_argv_mode     00000001800048c4 f   MSVCRT:argv_mode.obj
 0001:000038cc       __scrt_is_ucrt_dll_in_use  00000001800048cc f   MSVCRT:ucrt_detection.obj
 0001:000038e0       memcpy                     00000001800048e0 f   vcruntime:VCRUNTIME140.dll
 0001:000038e6       memset                     00000001800048e6 f   vcruntime:VCRUNTIME140.dll
 0001:000038ec       strchr                     00000001800048ec f   vcruntime:VCRUNTIME140.dll
 0001:000038f2       __C_specific_handler       00000001800048f2 f   vcruntime:VCRUNTIME140.dll
 0001:000038f8       __std_type_info_destroy_list 00000001800048f8 f   vcruntime:VCRUNTIME140.dll
 0001:000038fe       strcmp                     00000001800048fe f   ucrt:api-ms-win-crt-string-l1-1-0.dll
 0001:00003904       strlen                     0000000180004904 f   ucrt:api-ms-win-crt-string-l1-1-0.dll
 0001:0000390a       _initterm                  000000018000490a f   ucrt:api-ms-win-crt-runtime-l1-1-0.dll
 0001:00003910       _initterm_e                0000000180004910 f   ucrt:api-ms-win-crt-runtime-l1-1-0.dll
 0001:00003916       _seh_filter_dll            0000000180004916 f   ucrt:api-ms-win-crt-runtime-l1-1-0.dll
 0001:0000391c       _configure_narrow_argv     000000018000491c f   ucrt:api-ms-win-crt-runtime-l1-1-0.dll
 0001:00003922       _initialize_narrow_environment 0000000180004922 f   ucrt:api-ms-win-crt-runtime-l1-1-0.dll
 0001:00003928       _initialize_onexit_table   0000000180004928 f   ucrt:api-ms-win-crt-runtime-l1-1-0.dll
 0001:0000392e       _register_onexit_function  000000018000492e f   ucrt:api-ms-win-crt-runtime-l1-1-0.dll
 0001:00003934       _execute_onexit_table      0000000180004934 f   ucrt:api-ms-win-crt-runtime-l1-1-0.dll
 0001:0000393a       _crt_atexit                000000018000493a f   ucrt:api-ms-win-crt-runtime-l1-1-0.dll
 0001:00003940       _cexit                     0000000180004940 f   ucrt:api-ms-win-crt-runtime-l1-1-0.dll
 0001:00003948       __acrt_initialize          0000000180004948 f   MSVCRT:ucrt_stubs.obj
 0001:00003948       __acrt_thread_attach       0000000180004948 f   MSVCRT:ucrt_stubs.obj
 0001:00003948       __acrt_thread_detach       0000000180004948 f   MSVCRT:ucrt_stubs.obj
 0001:00003948       __acrt_uninitialize        0000000180004948 f   MSVCRT:ucrt_stubs.obj
 0001:00003948       __acrt_uninitialize_critical 0000000180004948 f   MSVCRT:ucrt_stubs.obj
 0001:00003948       __scrt_stub_for_acrt_initialize 0000000180004948 f   MSVCRT:ucrt_stubs.obj
 0001:00003948       __scrt_stub_for_acrt_thread_attach 0000000180004948 f   MSVCRT:ucrt_stubs.obj
 0001:00003948       __scrt_stub_for_acrt_thread_detach 0000000180004948 f   MSVCRT:ucrt_stubs.obj
 0001:00003948       __scrt_stub_for_acrt_uninitialize 0000000180004948 f   MSVCRT:ucrt_stubs.obj
 0001:00003948       __scrt_stub_for_acrt_uninitialize_critical 0000000180004948 f   MSVCRT:ucrt_stubs.obj
 0001:00003948       __vcrt_initialize          0000000180004948 f   MSVCRT:ucrt_stubs.obj
 0001:00003948       __vcrt_thread_attach       0000000180004948 f   MSVCRT:ucrt_stubs.obj
 0001:00003948       __vcrt_thread_detach       0000000180004948 f   MSVCRT:ucrt_stubs.obj
 0001:00003948       __vcrt_uninitialize        0000000180004948 f   MSVCRT:ucrt_stubs.obj
 0001:00003948       __vcrt_uninitialize_critical 0000000180004948 f   MSVCRT:ucrt_stubs.obj
 0001:0000394c       __scrt_stub_for_is_c_termination_complete 000000018000494c f   MSVCRT:ucrt_stubs.obj
 0001:0000394c       _is_c_termination_complete 000000018000494c f   MSVCRT:ucrt_stubs.obj
 0001:00003960       _guard_dispatch_icall_nop  0000000180004960 f   MSVCRT:guard_dispatch.obj
 0001:00003980       _guard_xfg_dispatch_icall_nop 0000000180004980 f   MSVCRT:guard_xfg_dispatch.obj
 0002:00000000       __imp_RtlCaptureContext    0000000180005000     kernel32:KERNEL32.dll
 0002:00000008       __imp_RtlLookupFunctionEntry 0000000180005008     kernel32:KERNEL32.dll
 0002:00000010       __imp_RtlVirtualUnwind     0000000180005010     kernel32:KERNEL32.dll
 0002:00000018       __imp_UnhandledExceptionFilter 0000000180005018     kernel32:KERNEL32.dll
 0002:00000020       __imp_SetUnhandledExceptionFilter 0000000180005020     kernel32:KERNEL32.dll
 0002:00000028       __imp_GetCurrentProcess    0000000180005028     kernel32:KERNEL32.dll
 0002:00000030       __imp_TerminateProcess     0000000180005030     kernel32:KERNEL32.dll
 0002:00000038       __imp_IsProcessorFeaturePresent 0000000180005038     kernel32:KERNEL32.dll
 0002:00000040       __imp_CloseHandle          0000000180005040     kernel32:KERNEL32.dll
 0002:00000048       __imp_InitializeCriticalSectionAndSpinCount 0000000180005048     kernel32:KERNEL32.dll
 0002:00000050       __imp_DeleteCriticalSection 0000000180005050     kernel32:KERNEL32.dll
 0002:00000058       __imp_CreateEventW         0000000180005058     kernel32:KERNEL32.dll
 0002:00000060       __imp_GetModuleHandleW     0000000180005060     kernel32:KERNEL32.dll
 0002:00000068       __imp_GetProcAddress       0000000180005068     kernel32:KERNEL32.dll
 0002:00000070       __imp_IsDebuggerPresent    0000000180005070     kernel32:KERNEL32.dll
 0002:00000078       __imp_QueryPerformanceCounter 0000000180005078     kernel32:KERNEL32.dll
 0002:00000080       __imp_GetCurrentProcessId  0000000180005080     kernel32:KERNEL32.dll
 0002:00000088       __imp_GetCurrentThreadId   0000000180005088     kernel32:KERNEL32.dll
 0002:00000090       __imp_GetSystemTimeAsFileTime 0000000180005090     kernel32:KERNEL32.dll
 0002:00000098       __imp_DisableThreadLibraryCalls 0000000180005098     kernel32:KERNEL32.dll
 0002:000000a0       __imp_InitializeSListHead  00000001800050a0     kernel32:KERNEL32.dll
 0002:000000a8       \177KERNEL32_NULL_THUNK_DATA 00000001800050a8     kernel32:KERNEL32.dll
 0002:000000b0       __imp_memcpy               00000001800050b0     vcruntime:VCRUNTIME140.dll
 0002:000000b8       __imp_memset               00000001800050b8     vcruntime:VCRUNTIME140.dll
 0002:000000c0       __imp_strchr               00000001800050c0     vcruntime:VCRUNTIME140.dll
 0002:000000c8       __imp___C_specific_handler 00000001800050c8     vcruntime:VCRUNTIME140.dll
 0002:000000d0       __imp___std_type_info_destroy_list 00000001800050d0     vcruntime:VCRUNTIME140.dll
 0002:000000d8       \177VCRUNTIME140_NULL_THUNK_DATA 00000001800050d8     vcruntime:VCRUNTIME140.dll
 0002:000000e0       __imp_strtol               00000001800050e0     ucrt:api-ms-win-crt-convert-l1-1-0.dll
 0002:000000e8       \177api-ms-win-crt-convert-l1-1-0_NULL_THUNK_DATA 00000001800050e8     ucrt:api-ms-win-crt-convert-l1-1-0.dll
 0002:000000f0       __imp_malloc               00000001800050f0     ucrt:api-ms-win-crt-heap-l1-1-0.dll
 0002:000000f8       __imp_free                 00000001800050f8     ucrt:api-ms-win-crt-heap-l1-1-0.dll
 0002:00000100       \177api-ms-win-crt-heap-l1-1-0_NULL_THUNK_DATA 0000000180005100     ucrt:api-ms-win-crt-heap-l1-1-0.dll
 0002:00000108       __imp__errno               0000000180005108     ucrt:api-ms-win-crt-runtime-l1-1-0.dll
 0002:00000110       __imp_exit                 0000000180005110     ucrt:api-ms-win-crt-runtime-l1-1-0.dll
 0002:00000118       __imp__cexit               0000000180005118     ucrt:api-ms-win-crt-runtime-l1-1-0.dll
 0002:00000120       __imp__crt_atexit          0000000180005120     ucrt:api-ms-win-crt-runtime-l1-1-0.dll
 0002:00000128       __imp__execute_onexit_table 0000000180005128     ucrt:api-ms-win-crt-runtime-l1-1-0.dll
 0002:00000130       __imp__register_onexit_function 0000000180005130     ucrt:api-ms-win-crt-runtime-l1-1-0.dll
 0002:00000138       __imp__initialize_onexit_table 0000000180005138     ucrt:api-ms-win-crt-runtime-l1-1-0.dll
 0002:00000140       __imp__initialize_narrow_environment 0000000180005140     ucrt:api-ms-win-crt-runtime-l1-1-0.dll
 0002:00000148       __imp__configure_narrow_argv 0000000180005148     ucrt:api-ms-win-crt-runtime-l1-1-0.dll
 0002:00000150       __imp__seh_filter_dll      0000000180005150     ucrt:api-ms-win-crt-runtime-l1-1-0.dll
 0002:00000158       __imp__initterm_e          0000000180005158     ucrt:api-ms-win-crt-runtime-l1-1-0.dll
 0002:00000160       __imp__initterm            0000000180005160     ucrt:api-ms-win-crt-runtime-l1-1-0.dll
 0002:00000168       \177api-ms-win-crt-runtime-l1-1-0_NULL_THUNK_DATA 0000000180005168     ucrt:api-ms-win-crt-runtime-l1-1-0.dll
 0002:00000170       __imp___acrt_iob_func      0000000180005170     ucrt:api-ms-win-crt-stdio-l1-1-0.dll
 0002:00000178       __imp_fflush               0000000180005178     ucrt:api-ms-win-crt-stdio-l1-1-0.dll
 0002:00000180       __imp___stdio_common_vsprintf 0000000180005180     ucrt:api-ms-win-crt-stdio-l1-1-0.dll
 0002:00000188       __imp___stdio_common_vfprintf 0000000180005188     ucrt:api-ms-win-crt-stdio-l1-1-0.dll
 0002:00000190       \177api-ms-win-crt-stdio-l1-1-0_NULL_THUNK_DATA 0000000180005190     ucrt:api-ms-win-crt-stdio-l1-1-0.dll
 0002:00000198       __imp_strcmp               0000000180005198     ucrt:api-ms-win-crt-string-l1-1-0.dll
 0002:000001a0       __imp__strdup              00000001800051a0     ucrt:api-ms-win-crt-string-l1-1-0.dll
 0002:000001a0       __imp_strdup               00000001800051a0     ucrt:api-ms-win-crt-string-l1-1-0.dll
 0002:000001a8       __imp_strlen               00000001800051a8     ucrt:api-ms-win-crt-string-l1-1-0.dll
 0002:000001b0       __imp_strpbrk              00000001800051b0     ucrt:api-ms-win-crt-string-l1-1-0.dll
 0002:000001b8       __imp_strncpy              00000001800051b8     ucrt:api-ms-win-crt-string-l1-1-0.dll
 0002:000001c0       \177api-ms-win-crt-string-l1-1-0_NULL_THUNK_DATA 00000001800051c0     ucrt:api-ms-win-crt-string-l1-1-0.dll
 0002:000001c8       __guard_check_icall_fptr   00000001800051c8     MSVCRT:guard_support.obj
 0002:000001d0       __guard_xfg_check_icall_fptr 00000001800051d0     MSVCRT:guard_support.obj
 0002:000001d8       __guard_dispatch_icall_fptr 00000001800051d8     MSVCRT:guard_support.obj
 0002:000001e0       __guard_xfg_dispatch_icall_fptr 00000001800051e0     MSVCRT:guard_support.obj
 0002:000001e8       __guard_xfg_table_dispatch_icall_fptr 00000001800051e8     MSVCRT:guard_support.obj
 0002:000001f0       __castguard_check_failure_os_handled_fptr 00000001800051f0     MSVCRT:guard_support.obj
 0002:000001f8       __guard_memcpy_fptr        00000001800051f8     vcruntime:softmemtag.obj
 0002:00000200       __xc_a                     0000000180005200     MSVCRT:initializers.obj
 0002:00000208       __xc_z                     0000000180005208     MSVCRT:initializers.obj
 0002:00000210       __xi_a                     0000000180005210     MSVCRT:initializers.obj
 0002:00000220       __xi_z                     0000000180005220     MSVCRT:initializers.obj
 0002:00000228       __xl_a                     0000000180005228     MSVCRT:tlssup.obj
 0002:00000230       __xl_z                     0000000180005230     MSVCRT:tlssup.obj
 0002:00000238       __xp_a                     0000000180005238     MSVCRT:initializers.obj
 0002:00000240       __xp_z                     0000000180005240     MSVCRT:initializers.obj
 0002:00000248       __xt_a                     0000000180005248     MSVCRT:initializers.obj
 0002:00000250       __xt_z                     0000000180005250     MSVCRT:initializers.obj
 0002:00000260       g_refKindStr               0000000180005260     libobjsize001.obj
 0002:00000410       ??_C@_09BPLDFGCI@unknown_0@ 0000000180005410     libobjsize001.obj
 0002:00000420       ??_C@_0BL@FPNMECJD@JVMTI_HEAP_REFERENCE_CLASS@ 0000000180005420     libobjsize001.obj
 0002:00000440       ??_C@_0BL@FKGKKLNM@JVMTI_HEAP_REFERENCE_FIELD@ 0000000180005440     libobjsize001.obj
 0002:00000460       ??_C@_0CD@CAEHCFJF@JVMTI_HEAP_REFERENCE_ARRAY_ELEM@ 0000000180005460     libobjsize001.obj
 0002:00000488       ??_C@_0CC@DNEBMCNK@JVMTI_HEAP_REFERENCE_CLASS_LOAD@ 0000000180005488     libobjsize001.obj
 0002:000004b0       ??_C@_0BN@CJMIPEBB@JVMTI_HEAP_REFERENCE_SIGNERS@ 00000001800054b0     libobjsize001.obj
 0002:000004d0       ??_C@_0CH@HBOIDPEB@JVMTI_HEAP_REFERENCE_PROTECTION@ 00000001800054d0     libobjsize001.obj
 0002:000004f8       ??_C@_0BP@MDKGDGKL@JVMTI_HEAP_REFERENCE_INTERFACE@ 00000001800054f8     libobjsize001.obj
 0002:00000518       ??_C@_0CC@JJMIHNJH@JVMTI_HEAP_REFERENCE_STATIC_FIE@ 0000000180005518     libobjsize001.obj
 0002:00000540       ??_C@_0CD@IDHEEGID@JVMTI_HEAP_REFERENCE_CONSTANT_P@ 0000000180005540     libobjsize001.obj
 0002:00000568       ??_C@_0CA@EFFCHNG@JVMTI_HEAP_REFERENCE_SUPERCLASS@ 0000000180005568     libobjsize001.obj
 0002:00000588       ??_C@_0L@PCDFHGCJ@unknown_11@ 0000000180005588     libobjsize001.obj
 0002:00000598       ??_C@_0L@NJBICFOK@unknown_12@ 0000000180005598     libobjsize001.obj
 0002:000005a8       ??_C@_0L@MAADBEKL@unknown_13@ 00000001800055a8     libobjsize001.obj
 0002:000005b8       ??_C@_0L@IPECICGM@unknown_14@ 00000001800055b8     libobjsize001.obj
 0002:000005c8       ??_C@_0L@JGFJLDCN@unknown_15@ 00000001800055c8     libobjsize001.obj
 0002:000005d8       ??_C@_0L@LNHEOAOO@unknown_16@ 00000001800055d8     libobjsize001.obj
 0002:000005e8       ??_C@_0L@KEGPNBKP@unknown_17@ 00000001800055e8     libobjsize001.obj
 0002:000005f8       ??_C@_0L@CDPHMNGA@unknown_18@ 00000001800055f8     libobjsize001.obj
 0002:00000608       ??_C@_0L@DKOMPMCB@unknown_19@ 0000000180005608     libobjsize001.obj
 0002:00000618       ??_C@_0L@OJGIPJDB@unknown_20@ 0000000180005618     libobjsize001.obj
 0002:00000628       ??_C@_0CA@KAOFNDEM@JVMTI_HEAP_REFERENCE_JNI_GLOBAL@ 0000000180005628     libobjsize001.obj
 0002:00000648       ??_C@_0CC@HPFAJBK@JVMTI_HEAP_REFERENCE_SYSTEM_CLA@ 0000000180005648     libobjsize001.obj
 0002:00000670       ??_C@_0BN@FDEGFOHC@JVMTI_HEAP_REFERENCE_MONITOR@ 0000000180005670     libobjsize001.obj
 0002:00000690       ??_C@_0CB@HKIBCMAJ@JVMTI_HEAP_REFERENCE_STACK_LOCA@ 0000000180005690     libobjsize001.obj
 0002:000006b8       ??_C@_0BP@EAACMMOE@JVMTI_HEAP_REFERENCE_JNI_LOCAL@ 00000001800056b8     libobjsize001.obj
 0002:000006d8       ??_C@_0BM@IJDEOGOE@JVMTI_HEAP_REFERENCE_THREAD@ 00000001800056d8     libobjsize001.obj
 0002:000006f8       ??_C@_0BL@EDGPPKC@JVMTI_HEAP_REFERENCE_OTHER@ 00000001800056f8     libobjsize001.obj
 0002:00000714       ??_C@_04BCJPDBDA@Code@     0000000180005714     libobjsize001.obj
 0002:00000720       ??_C@_0BA@OCLMCFKC@LineNumberTable@ 0000000180005720     libobjsize001.obj
 0002:00000730       ??_C@_0BD@CPAEPILC@LocalVariableTable@ 0000000180005730     libobjsize001.obj
 0002:00000748       ??_C@_0BH@NMBDNHBD@LocalVariableTypeTable@ 0000000180005748     libobjsize001.obj
 0002:00000760       ??_C@_0O@HIHEEDNJ@StackMapTable@ 0000000180005760     libobjsize001.obj
 0002:00000770       ??_C@_0L@HCDIAMJG@?9?5?$CFs?0?5?$CFd?3?5@ 0000000180005770     libobjsize001.obj
 0002:00000780       ??_C@_0JI@HLPECLFI@?$CD?5?4?4?4?6?$CD?5ERROR?3?5too?5many?5complai@ 0000000180005780     libobjsize001.obj
 0002:00000820       ??_C@_0ED@JNEKCCOB@The?5following?5fake?5exception?5st@ 0000000180005820     libobjsize001.obj
 0002:00000868       ??_C@_0CN@FCNMDFBH@nsk?4share?4Fake_Exception_for_RU@ 0000000180005868     libobjsize001.obj
 0002:00000898       ??_C@_08PGFFNAEI@?$CI?$CFs?3?$CFd?$CJ?5@ 0000000180005898     libobjsize001.obj
 0002:000008a8       ??_C@_0DP@IENMAEGI@s?2test?2hotspot?2jtreg?2vmTestbase@ 00000001800058a8     libobjsize001.obj
 0002:000008e8       ??_C@_0BL@NDJLFFJB@?7at?5nsk_lvcomplain?$CI?$CFs?3?$CFd?$CJ?6@ 00000001800058e8     libobjsize001.obj
 0002:00000908       ??_C@_0BC@JOOKAFKF@?$CD?5ERROR?3?5?$CFs?0?5?$CFd?3?5@ 0000000180005908     libobjsize001.obj
 0002:00000920       ??_C@_09KJEAHMEH@?$CD?5ERROR?3?5@ 0000000180005920     libobjsize001.obj
 0002:0000092c       ??_C@_02GPIOPFAK@?$DO?$DO@ 000000018000592c     libobjsize001.obj
 0002:00000930       ??_C@_02FODMEDOG@?$DM?$DM@ 0000000180005930     libobjsize001.obj
 0002:00000934       ??_C@_02DJGKEECL@?4?4@     0000000180005934     libobjsize001.obj
 0002:00000938       ??_C@_0O@CJPGJOAF@?9?5?$CFs?0?5?$CFd?3?5?$CFs?5@ 0000000180005938     libobjsize001.obj
 0002:00000948       ??_C@_0CB@IAKPDOIC@?$CD?5?5?5verified?5assertion?5is?5FALSE@ 0000000180005948     libobjsize001.obj
 0002:00000970       ??_C@_0CO@LGONDEPD@stdout?3?5fflush?5failed?5?9?5err?$DN?$CFd?5@ 0000000180005970     libobjsize001.obj
 0002:000009a0       ??_C@_0CO@KBGKJPBD@stderr?3?5fflush?5failed?5?9?5err?$DN?$CFd?5@ 00000001800059a0     libobjsize001.obj
 0002:000009d0       ??_C@_0BB@JCNMKLLK@JVMTI_ERROR_NONE@ 00000001800059d0     libobjsize001.obj
 0002:000009e8       ??_C@_0BL@LDIMKLPH@JVMTI_ERROR_INVALID_THREAD@ 00000001800059e8     libobjsize001.obj
 0002:00000a08       ??_C@_0CB@PJFPAIKJ@JVMTI_ERROR_INVALID_THREAD_GROU@ 0000000180005a08     libobjsize001.obj
 0002:00000a30       ??_C@_0BN@LLMKHMNF@JVMTI_ERROR_INVALID_PRIORITY@ 0000000180005a30     libobjsize001.obj
 0002:00000a50       ??_C@_0CB@MBOFKAGB@JVMTI_ERROR_THREAD_NOT_SUSPENDE@ 0000000180005a50     libobjsize001.obj
 0002:00000a78       ??_C@_0BN@FABOLPBI@JVMTI_ERROR_THREAD_SUSPENDED@ 0000000180005a78     libobjsize001.obj
 0002:00000a98       ??_C@_0BN@FDGNOBJM@JVMTI_ERROR_THREAD_NOT_ALIVE@ 0000000180005a98     libobjsize001.obj
 0002:00000ab8       ??_C@_0BL@GOBIFKNJ@JVMTI_ERROR_INVALID_OBJECT@ 0000000180005ab8     libobjsize001.obj
 0002:00000ad8       ??_C@_0BK@FCMAJPPC@JVMTI_ERROR_INVALID_CLASS@ 0000000180005ad8     libobjsize001.obj
 0002:00000af8       ??_C@_0BP@IKLLBKEB@JVMTI_ERROR_CLASS_NOT_PREPARED@ 0000000180005af8     libobjsize001.obj
 0002:00000b18       ??_C@_0BN@KLPPLKG@JVMTI_ERROR_INVALID_METHODID@ 0000000180005b18     libobjsize001.obj
 0002:00000b38       ??_C@_0BN@BCEKOKND@JVMTI_ERROR_INVALID_LOCATION@ 0000000180005b38     libobjsize001.obj
 0002:00000b58       ??_C@_0BM@DFDGPME@JVMTI_ERROR_INVALID_FIELDID@ 0000000180005b58     libobjsize001.obj
 0002:00000b78       ??_C@_0BL@NELIEPEC@JVMTI_ERROR_NO_MORE_FRAMES@ 0000000180005b78     libobjsize001.obj
 0002:00000b98       ??_C@_0BJ@BDBECFDM@JVMTI_ERROR_OPAQUE_FRAME@ 0000000180005b98     libobjsize001.obj
 0002:00000bb8       ??_C@_0BK@MIIFNLOB@JVMTI_ERROR_TYPE_MISMATCH@ 0000000180005bb8     libobjsize001.obj
 0002:00000bd8       ??_C@_0BJ@HPCAOILC@JVMTI_ERROR_INVALID_SLOT@ 0000000180005bd8     libobjsize001.obj
 0002:00000bf8       ??_C@_0BG@CHILOPNI@JVMTI_ERROR_DUPLICATE@ 0000000180005bf8     libobjsize001.obj
 0002:00000c10       ??_C@_0BG@DIEMLHKM@JVMTI_ERROR_NOT_FOUND@ 0000000180005c10     libobjsize001.obj
 0002:00000c28       ??_C@_0BM@NHMCKHOB@JVMTI_ERROR_INVALID_MONITOR@ 0000000180005c28     libobjsize001.obj
 0002:00000c48       ??_C@_0BO@PPEDAJGL@JVMTI_ERROR_NOT_MONITOR_OWNER@ 0000000180005c48     libobjsize001.obj
 0002:00000c68       ??_C@_0BG@FCAIPEID@JVMTI_ERROR_INTERRUPT@ 0000000180005c68     libobjsize001.obj
 0002:00000c80       ??_C@_0CB@EGDBNKOI@JVMTI_ERROR_INVALID_CLASS_FORMA@ 0000000180005c80     libobjsize001.obj
 0002:00000ca8       ??_C@_0CG@DGKOGIAL@JVMTI_ERROR_CIRCULAR_CLASS_DEFI@ 0000000180005ca8     libobjsize001.obj
 0002:00000cd0       ??_C@_0BP@ICEALPKC@JVMTI_ERROR_FAILS_VERIFICATION@ 0000000180005cd0     libobjsize001.obj
 0002:00000cf0       ??_C@_0DC@JDACLMIO@JVMTI_ERROR_UNSUPPORTED_REDEFIN@ 0000000180005cf0     libobjsize001.obj
 0002:00000d28       ??_C@_0DE@GKDKNOMJ@JVMTI_ERROR_UNSUPPORTED_REDEFIN@ 0000000180005d28     libobjsize001.obj
 0002:00000d60       ??_C@_0BO@LAFKIOG@JVMTI_ERROR_INVALID_TYPESTATE@ 0000000180005d60     libobjsize001.obj
 0002:00000d80       ??_C@_0DH@INDGCLLB@JVMTI_ERROR_UNSUPPORTED_REDEFIN@ 0000000180005d80     libobjsize001.obj
 0002:00000db8       ??_C@_0DE@NHEOMMGI@JVMTI_ERROR_UNSUPPORTED_REDEFIN@ 0000000180005db8     libobjsize001.obj
 0002:00000df0       ??_C@_0CA@EKPNJOEP@JVMTI_ERROR_UNSUPPORTED_VERSION@ 0000000180005df0     libobjsize001.obj
 0002:00000e10       ??_C@_0BN@OFFMAHHL@JVMTI_ERROR_NAMES_DONT_MATCH@ 0000000180005e10     libobjsize001.obj
 0002:00000e30       ??_C@_0DN@HHBBLAKE@JVMTI_ERROR_UNSUPPORTED_REDEFIN@ 0000000180005e30     libobjsize001.obj
 0002:00000e70       ??_C@_0DO@HMBGBGNA@JVMTI_ERROR_UNSUPPORTED_REDEFIN@ 0000000180005e70     libobjsize001.obj
 0002:00000eb0       ??_C@_0BP@PBECGKHJ@JVMTI_ERROR_UNMODIFIABLE_CLASS@ 0000000180005eb0     libobjsize001.obj
 0002:00000ed0       ??_C@_0BK@CANILEHF@JVMTI_ERROR_NOT_AVAILABLE@ 0000000180005ed0     libobjsize001.obj
 0002:00000ef0       ??_C@_0CE@INJKMEFK@JVMTI_ERROR_MUST_POSSESS_CAPABI@ 0000000180005ef0     libobjsize001.obj
 0002:00000f18       ??_C@_0BJ@LBFPFPDM@JVMTI_ERROR_NULL_POINTER@ 0000000180005f18     libobjsize001.obj
 0002:00000f38       ??_C@_0BP@CHJPNNEM@JVMTI_ERROR_ABSENT_INFORMATION@ 0000000180005f38     libobjsize001.obj
 0002:00000f58       ??_C@_0BP@OMFMNLC@JVMTI_ERROR_INVALID_EVENT_TYPE@ 0000000180005f58     libobjsize001.obj
 0002:00000f78       ??_C@_0BN@BIBNPHHO@JVMTI_ERROR_ILLEGAL_ARGUMENT@ 0000000180005f78     libobjsize001.obj
 0002:00000f98       ??_C@_0BK@KKNDHDCE@JVMTI_ERROR_NATIVE_METHOD@ 0000000180005f98     libobjsize001.obj
 0002:00000fb8       ??_C@_0BK@PMKCFHAE@JVMTI_ERROR_OUT_OF_MEMORY@ 0000000180005fb8     libobjsize001.obj
 0002:00000fd8       ??_C@_0BK@NNJBDMNB@JVMTI_ERROR_ACCESS_DENIED@ 0000000180005fd8     libobjsize001.obj
 0002:00000ff8       ??_C@_0BI@GHECLMNC@JVMTI_ERROR_WRONG_PHASE@ 0000000180005ff8     libobjsize001.obj
 0002:00001010       ??_C@_0BF@OLIHJOII@JVMTI_ERROR_INTERNAL@ 0000000180006010     libobjsize001.obj
 0002:00001028       ??_C@_0BO@EOHGKJHI@JVMTI_ERROR_UNATTACHED_THREAD@ 0000000180006028     libobjsize001.obj
 0002:00001048       ??_C@_0CA@LKHFDACL@JVMTI_ERROR_INVALID_ENVIRONMENT@ 0000000180006048     libobjsize001.obj
 0002:00001068       ??_C@_0BA@MMFHLOKK@?$DMunknown?5error?$DO@ 0000000180006068     libobjsize001.obj
 0002:00001078       ??_C@_0CF@CBHOKDB@throwable?5?$DN?5jni?9?$DOExceptionOccur@ 0000000180006078     libobjsize001.obj
 0002:000010a0       ??_C@_03OFAPEBGM@?$CFs?6@  00000001800060a0     libobjsize001.obj
 0002:000010a8       ??_C@_0DM@LPIGEGNJ@s?2test?2hotspot?2jtreg?2vmTestbase@ 00000001800060a8     libobjsize001.obj
 0002:000010e8       ??_C@_0CC@NFCNPEPK@Exception?5in?5JNI?5call?5?$CIcleared?$CJ@ 00000001800060e8     libobjsize001.obj
 0002:00001110       ??_C@_0BJ@IBAKFIKF@jni?9?$DOExceptionDescribe?$CI?$CJ@ 0000000180006110     libobjsize001.obj
 0002:00001130       ??_C@_0BG@GGKALKMH@jni?9?$DOExceptionClear?$CI?$CJ@ 0000000180006130     libobjsize001.obj
 0002:00001148       ??_C@_0CF@JMGFGJLJ@?$CD?5?5?5verified?5JNI?5assertion?5is?5F@ 0000000180006148     libobjsize001.obj
 0002:00001170       ??_C@_07KBAMPNJK@verbose@  0000000180006170     libobjsize001.obj
 0002:00001178       ??_C@_0DN@PKJBOLAP@nsk_jvmti_parseOptions?$CI?$CJ?3?5unexp@ 0000000180006178     libobjsize001.obj
 0002:000011b8       ??_C@_05IMBNNINJ@trace@    00000001800061b8     libobjsize001.obj
 0002:000011c0       ??_C@_0DD@BJKGNDMB@nsk_jvmti_parseOptions?$CI?$CJ?3?5no?5va@ 00000001800061c0     libobjsize001.obj
 0002:000011f4       ??_C@_04CGFJFPFD@none@     00000001800061f4     libobjsize001.obj
 0002:000011fc       ??_C@_06BMELKFMA@before@   00000001800061fc     libobjsize001.obj
 0002:00001204       ??_C@_05CMKPCFDK@after@    0000000180006204     libobjsize001.obj
 0002:0000120c       ??_C@_03NFKEKGGK@all@      000000018000620c     libobjsize001.obj
 0002:00001210       ??_C@_0DM@NDNJGJKE@nsk_jvmti_parseOptions?$CI?$CJ?3?5uexpe@ 0000000180006210     libobjsize001.obj
 0002:00001250       ??_C@_08NBBJKJO@waittime@  0000000180006250     libobjsize001.obj
 0002:00001260       ??_C@_0DO@CMHGAOHC@nsk_jvmti_parseOptions?$CI?$CJ?3?5not?5i@ 0000000180006260     libobjsize001.obj
 0002:000012a0       ??_C@_0DL@LNMPBDLN@nsk_jvmti_parseOptions?$CI?$CJ?3?5negat@ 00000001800062a0     libobjsize001.obj
 0002:000012e0       ??_C@_0DA@GMFJNOJH@nsk_jvmti_parseOptions?$CI?$CJ?3?5unkno@ 00000001800062e0     libobjsize001.obj
 0002:00001310       ??_C@_0CO@CCIAMEAN@nsk_jvmti_parseOptions?$CI?$CJ?3?5found@ 0000000180006310     libobjsize001.obj
 0002:00001340       ??_C@_0CJ@OEGPCGDL@nsk_jvmti_parseOptions?$CI?$CJ?3?5out?5o@ 0000000180006340     libobjsize001.obj
 0002:00001370       ??_C@_0DI@NMBHPGGF@nsk_jvmti_parseOptions?$CI?$CJ?3?5too?5m@ 0000000180006370     libobjsize001.obj
 0002:000013a8       ??_C@_03POGCGECB@?5?0?$HO@ 00000001800063a8     libobjsize001.obj
 0002:000013b0       ??_C@_0CB@MLNJNCLJ@?5?5jvmti?5error?3?5code?$DN?$CFd?0?5name?$DN?$CFs@ 00000001800063b0     libobjsize001.obj
 0002:000013d8       ??_C@_0CD@OHBGDKMK@?$CD?5?5?5jvmti?5error?3?5code?$DN?$CFd?0?5name?$DN@ 00000001800063d8     libobjsize001.obj
 0002:00001400       ??_C@_0CG@JNNCGPHB@?$CD?5?5?5error?5expected?3?5code?$DN?$CFd?0?5na@ 0000000180006400     libobjsize001.obj
 0002:00001430       ??_C@_0EB@IMGKPCGE@?$CIstr_obj?5?$DN?5jni?9?$DONewStringUTF?$CIco@ 0000000180006430     libobjsize001.obj
 0002:00001480       ??_C@_0EA@HFOGGBCC@s?2test?2hotspot?2jtreg?2vmTestbase@ 0000000180006480     libobjsize001.obj
 0002:000014c0       ??_C@_05KKCIMGE@error@     00000001800064c0     libobjsize001.obj
 0002:000014c8       ??_C@_0CJ@JACLEAA@Test?5failed?5by?5setFailStatus?$CI?$CJ?4@ 00000001800064c8     libobjsize001.obj
 0002:000014f8       ??_C@_0BD@HGNAOMCP@agent_data_monitor@ 00000001800064f8     libobjsize001.obj
 0002:00001510       ??_C@_0EB@OGCLGKLN@javaVM?9?$DOGetEnv?$CI?$CIvoid?5?$CK?$CK?$CJ?$CGjvmti_@ 0000000180006510     libobjsize001.obj
 0002:00001560       ??_C@_0EA@PNBCDMOA@s?2test?2hotspot?2jtreg?2vmTestbase@ 0000000180006560     libobjsize001.obj
 0002:000015a0       ??_C@_0CI@DDPIFBGM@init_agent_data?$CIjvmti_env?0?5?$CGage@ 00000001800065a0     libobjsize001.obj
 0002:000015c8       ??_C@_0DI@ILAHDLMP@?$CI?$CKagentThreadProc?$CJ?$CIjvmti_env?0?5a@ 00000001800065c8     libobjsize001.obj
 0002:00001600       ??_C@_0BD@KDBALNLB@JVMTI?5agent?5thread@ 0000000180006600     libobjsize001.obj
 0002:00001618       ??_C@_0BB@NOKBFPFO@java?1lang?1Thread@ 0000000180006618     libobjsize001.obj
 0002:0000162c       ??_C@_06FALKBLGB@?$DMinit?$DO@ 000000018000662c     libobjsize001.obj
 0002:00001638       ??_C@_0BG@IKDDPPGD@?$CILjava?1lang?1String?$DL?$CJV@ 0000000180006638     libobjsize001.obj
 0002:00001650       ??_C@_0EB@IFJBFEKC@?$CIthreadClass?5?$DN?5jni_env?9?$DOFindCla@ 0000000180006650     libobjsize001.obj
 0002:000016a0       ??_C@_0GF@FGFIBKKL@?$CIthreadCtor?5?$DN?5jni_env?9?$DOGetMetho@ 00000001800066a0     libobjsize001.obj
 0002:00001708       ??_C@_0DN@NCPDJLOG@?$CIthreadName?5?$DN?5jni_env?9?$DONewStrin@ 0000000180006708     libobjsize001.obj
 0002:00001750       ??_C@_0FE@PFKODBGC@?$CIthreadObject?5?$DN?5jni_env?9?$DONewObj@ 0000000180006750     libobjsize001.obj
 0002:000017b0       ??_C@_0ED@HOBAHHJI@?$CIthreadGlobalRef?5?$DN?5jni_env?9?$DONew@ 00000001800067b0     libobjsize001.obj
 0002:00001800       ??_C@_0FN@HNJJAHFC@jvmti_env?9?$DORunAgentThread?$CIagent@ 0000000180006800     libobjsize001.obj
 0002:00001860       ??_C@_0EA@MOJDNKDF@Debuggee?5status?5sync?5aborted?5be@ 0000000180006860     libobjsize001.obj
 0002:000018a0       ??_C@_0CO@PGPGMHBJ@No?5status?5sync?5occured?5for?5time@ 00000001800068a0     libobjsize001.obj
 0002:000018d0       ??_C@_0CL@DOEBDPKJ@Debuggee?5was?5not?5suspended?5on?5s@ 00000001800068d0     libobjsize001.obj
 0002:00001900       ??_C@_0EA@EEOEJAEN@status?5?$DN?5syncDebuggeeStatus?$CIjni@ 0000000180006900     libobjsize001.obj
 0002:00001940       ??_C@_0BL@JBCFNBMB@nsk_jvmti_resetAgentData?$CI?$CJ@ 0000000180006940     libobjsize001.obj
 0002:00001960       ??_C@_0EL@LPBEELIP@s?2test?2hotspot?2jtreg?2vmTestbase@ 0000000180006960     libobjsize001.obj
 0002:000019b0       ??_C@_0CK@JDAMFDMJ@jvmti?9?$DOSetTag?$CIo?0?5tag?$CJ?5?$DN?$DN?5JVMTI_@ 00000001800069b0     libobjsize001.obj
 0002:000019e0       ??_C@_0CC@DAMNHKNI@Can?8t?5set?5tag?5?$CFli?5for?5object?5?$CFl@ 00000001800069e0     libobjsize001.obj
 0002:00001a08       ??_C@_0DL@HAJPNKEF@jvmti?9?$DOGetObjectHashCode?$CIo?0?5?$CGha@ 0000000180006a08     libobjsize001.obj
 0002:00001a48       ??_C@_0BL@JFPIEOBF@Can?8t?5get?5hash?5object?5?$CFlx?6@ 0000000180006a48     libobjsize001.obj
 0002:00001a68       ??_C@_0BG@DICPHBKN@setTag?3?5?$CF08x?5?$DM?9?5?$CF?53li@ 0000000180006a68     libobjsize001.obj
 0002:00001a80       ??_C@_0DH@FCEEBDMJ@?$CIs?5?$DN?5jni?9?$DOGetStringUTFChars?$CIsIn@ 0000000180006a80     libobjsize001.obj
 0002:00001ab8       ??_C@_0BJ@OKKGHDCN@Can?8t?5get?5string?5at?5?$CF?$CDp?6@ 0000000180006ab8     libobjsize001.obj
 0002:00001ad8       ??_C@_0BP@EKFLGGFJ@Can?8t?5get?5string?5at?5?$CF?$CDp?3?5null?6@ 0000000180006ad8     libobjsize001.obj
 0002:00001af8       ??_C@_06ICODBHCL@?5?1?1?5?$CFs@ 0000000180006af8     libobjsize001.obj
 0002:00001b00       ??_C@_0DB@KGFPLEGO@?$CIr?5?$DN?5jvmti?9?$DOGetTag?$CIo?0?5?$CGtag?$CJ?$CJ?5?$DN?$DN@ 0000000180006b00     libobjsize001.obj
 0002:00001b38       ??_C@_0CO@PDAGBCGJ@Can?8t?5GetTag?5for?5object?5?$CFlx?4?5Re@ 0000000180006b38     libobjsize001.obj
 0002:00001b68       ??_C@_0CH@HPEODOHC@TEST_BUG?3?5Max?4?5number?5of?5refs?5r@ 0000000180006b68     libobjsize001.obj
 0002:00001b90       ??_C@_0DI@PHFCABIM@?$CIr?5?$DN?5jvmti?9?$DOGetTag?$CIfrom?0?5?$CGtagFr@ 0000000180006b90     libobjsize001.obj
 0002:00001bc8       ??_C@_0DI@MDEGFNKD@TEST_BUG?3?5Can?8t?5GetTag?5for?5obje@ 0000000180006bc8     libobjsize001.obj
 0002:00001c00       ??_C@_0DE@MLELJAHM@?$CIr?5?$DN?5jvmti?9?$DOGetTag?$CIto?0?5?$CGtagTo?$CJ?$CJ@ 0000000180006c00     libobjsize001.obj
 0002:00001c38       ??_C@_0BJ@NFJNGNHL@Wait?5for?5object?5created?6@ 0000000180006c38     libobjsize001.obj
 0002:00001c60       ??_C@_0FC@OFPNCJMI@s?2test?2hotspot?2jtreg?2vmTestbase@ 0000000180006c60     libobjsize001.obj
 0002:00001cb8       ??_C@_0BP@LAIJOMPC@nsk_jvmti_waitForSync?$CItimeout?$CJ@ 0000000180006cb8     libobjsize001.obj
 0002:00001cd8       ??_C@_0DP@LEBKMFGA@?$DO?$DO?$DO?5Obtain?5tested?5object?5from?5a@ 0000000180006cd8     libobjsize001.obj
 0002:00001d18       ??_C@_0CD@CEBDFMFM@nsk?1jvmti?1GetObjectSize?1objsize@ 0000000180006d18     libobjsize001.obj
 0002:00001d40       ??_C@_0BI@ENEOJHP@Find?5debugee?5class?3?5?$CFs?6@ 0000000180006d40     libobjsize001.obj
 0002:00001d58       ??_C@_0DP@MFMMLPOM@?$CIdebugeeClass?5?$DN?5jni?9?$DOFindClass?$CI@ 0000000180006d58     libobjsize001.obj
 0002:00001d98       ??_C@_0BJ@DFGCANJI@?5?5?4?4?4?5found?5class?3?50x?$CFp?6@ 0000000180006d98     libobjsize001.obj
 0002:00001db8       ??_C@_0N@MJMHMFFK@testedObject@ 0000000180006db8     libobjsize001.obj
 0002:00001dc8       ??_C@_0BH@PMPIFENK@Find?5static?5field?3?5?$CFs?6@ 0000000180006dc8     libobjsize001.obj
 0002:00001de0       ??_C@_0GE@KBCAFDGP@?$CIobjectField?5?$DN?5jni?9?$DOGetStaticFi@ 0000000180006de0     libobjsize001.obj
 0002:00001e48       ??_C@_0DA@PNEGIMGM@Lnsk?1jvmti?1GetObjectSize?1objsiz@ 0000000180006e48     libobjsize001.obj
 0002:00001e78       ??_C@_0BJ@MIIADDIH@?5?5?4?4?4?5got?5fieldID?3?50x?$CFp?6@ 0000000180006e78     libobjsize001.obj
 0002:00001e98       ??_C@_0CC@CDBPBOEE@Get?5object?5from?5static?5field?3?5?$CF@ 0000000180006e98     libobjsize001.obj
 0002:00001ec0       ??_C@_0FB@HNDBNKBP@?$CItestedObject?5?$DN?5jni?9?$DOGetStaticO@ 0000000180006ec0     libobjsize001.obj
 0002:00001f18       ??_C@_0BI@FNLCMIKO@?5?5?4?4?4?5got?5object?3?50x?$CFp?6@ 0000000180006f18     libobjsize001.obj
 0002:00001f30       ??_C@_0CK@DKJEDDCM@Create?5global?5reference?5for?5obj@ 0000000180006f30     libobjsize001.obj
 0002:00001f60       ??_C@_0DM@IGPAGPML@?$CItestedObject?5?$DN?5jni?9?$DONewGlobalR@ 0000000180006f60     libobjsize001.obj
 0002:00001fa0       ??_C@_0BL@LPHCNAPN@?5?5?4?4?4?5got?5reference?3?50x?$CFp?6@ 0000000180006fa0     libobjsize001.obj
 0002:00001fc0       ??_C@_0DB@HHOALPA@?$DO?$DO?$DO?5Testcase?5?$CD1?3?5get?5initial?5si@ 0000000180006fc0     libobjsize001.obj
 0002:00001ff8       ??_C@_0BL@HBCPOGMO@Get?5size?5for?5object?3?50x?$CFp?6@ 0000000180006ff8     libobjsize001.obj
 0002:00002018       ??_C@_0DA@LEAJLFH@jvmti?9?$DOGetObjectSize?$CItestedObje@ 0000000180007018     libobjsize001.obj
 0002:00002048       ??_C@_0CC@JGCCLDCG@?5?5?4?4?4?5got?5object?5size?3?5?$CFld?5byte@ 0000000180007048     libobjsize001.obj
 0002:00002070       ??_C@_0DP@FILJNLBK@GetObjectSize?$CI?$CJ?5returned?5unexpe@ 0000000180007070     libobjsize001.obj
 0002:000020b0       ??_C@_0EK@IMECBEB@?$DO?$DO?$DO?5Testcase?5?$CD2?3?5get?5size?5of?5no@ 00000001800070b0     libobjsize001.obj
 0002:00002100       ??_C@_0CK@GAMKPMJM@jvmti?9?$DOGetObjectSize?$CItestedObje@ 0000000180007100     libobjsize001.obj
 0002:00002130       ??_C@_0CC@LCHCLCIG@?5?5?4?4?4?5got?5object?5size?3?5?$CFld?6?5byt@ 0000000180007130     libobjsize001.obj
 0002:00002160       ??_C@_0IJ@CABEFIGJ@?$CD?5WARNING?3?5Other?5call?5to?5GetObj@ 0000000180007160     libobjsize001.obj
 0002:000021f0       ??_C@_0DJ@BPDDHLEB@SUCCESS?3?5Got?5object?5size?5is?5equ@ 00000001800071f0     libobjsize001.obj
 0002:00002230       ??_C@_0EG@PPCFFBFC@?$DO?$DO?$DO?5Testcase?5?$CD3?3?5get?5size?5of?5ch@ 0000000180007230     libobjsize001.obj
 0002:00002278       ??_C@_0CD@FIPENNEI@Let?5debugee?5to?5change?5object?5da@ 0000000180007278     libobjsize001.obj
 0002:000022a0       ??_C@_0BH@LECMGIIA@nsk_jvmti_resumeSync?$CI?$CJ@ 00000001800072a0     libobjsize001.obj
 0002:000022b8       ??_C@_0BM@DPJENODC@?5?5?4?4?4?5got?5object?5size?3?5?$CFld?6@ 00000001800072b8     libobjsize001.obj
 0002:000022e0       ??_C@_0IF@LCJNKEHB@?$CD?5WARNING?3?5Other?5call?5to?5GetObj@ 00000001800072e0     libobjsize001.obj
 0002:00002368       ??_C@_0BF@MNKEFEOE@?$DO?$DO?$DO?5Clean?5used?5data?6@ 0000000180007368     libobjsize001.obj
 0002:00002380       ??_C@_0BP@NCFBGLMD@Delete?5object?5reference?3?50x?$CFp?6@ 0000000180007380     libobjsize001.obj
 0002:000023a0       ??_C@_0CD@EIIDHGCH@jni?9?$DODeleteGlobalRef?$CItestedObje@ 00000001800073a0     libobjsize001.obj
 0002:000023c8       ??_C@_0BH@HPEOJMHL@Let?5debugee?5to?5finish?6@ 00000001800073c8     libobjsize001.obj
 0002:000023e0       ??_C@_0CA@MNKGCBCG@nsk_jvmti_parseOptions?$CIoptions?$CJ@ 00000001800073e0     libobjsize001.obj
 0002:00002400       ??_C@_0DN@MIAMNFPH@?$CIjvmti?5?$DN?5nsk_jvmti_createJVMTIE@ 0000000180007400     libobjsize001.obj
 0002:00002440       ??_C@_0CL@PIACJIPK@nsk_jvmti_setAgentProc?$CIagentPro@ 0000000180007440     libobjsize001.obj
 0002:00002480       ??_C@_1EC@JIJBPKFM@?$AAa?$AAp?$AAi?$AA?9?$AAm?$AAs?$AA?9?$AAw?$AAi?$AAn?$AA?9?$AAc?$AAo?$AAr?$AAe@ 0000000180007480     MSVCRT:thread_safe_statics.obj
 0002:000024c8       ??_C@_1BK@MGMFAEKH@?$AAk?$AAe?$AAr?$AAn?$AAe?$AAl?$AA3?$AA2?$AA?4?$AAd?$AAl?$AAl@ 00000001800074c8     MSVCRT:thread_safe_statics.obj
 0002:000024e8       ??_C@_0BJ@JEBJOJFJ@SleepConditionVariableCS@ 00000001800074e8     MSVCRT:thread_safe_statics.obj
 0002:00002508       ??_C@_0BJ@PGPPEPCC@WakeAllConditionVariable@ 0000000180007508     MSVCRT:thread_safe_statics.obj
 0002:00002528       _pDefaultRawDllMain        0000000180007528     MSVCRT:dll_dllmain.obj
 0002:00002528       _pRawDllMain               0000000180007528     MSVCRT:dll_dllmain.obj
 0002:00002530       __xmm@ffffffffffffffffffffffffffffffff 0000000180007530     MSVCRT:utility.obj
 0002:00002540       _load_config_used          0000000180007540     MSVCRT:loadcfg.obj
 0002:00002700       _tls_used                  0000000180007700     MSVCRT:tlssup.obj
 0002:00002728       __volatile_metadata        0000000180007728     <linker-defined>
 0002:00002b00       __rtc_iaa                  0000000180007b00     MSVCRT:initsect.obj
 0002:00002b08       __rtc_izz                  0000000180007b08     MSVCRT:initsect.obj
 0002:00002b10       __rtc_taa                  0000000180007b10     MSVCRT:initsect.obj
 0002:00002b18       __rtc_tzz                  0000000180007b18     MSVCRT:initsect.obj
 0002:00002b20       _tls_start                 0000000180007b20     MSVCRT:tlssup.obj
 0002:00002b24       _Init_thread_epoch         0000000180007b24     MSVCRT:thread_safe_statics.obj
 0002:00002b28       _tls_end                   0000000180007b28     MSVCRT:tlssup.obj
 0002:000031d4       __IMPORT_DESCRIPTOR_KERNEL32 00000001800081d4     kernel32:KERNEL32.dll
 0002:000031e8       __IMPORT_DESCRIPTOR_VCRUNTIME140 00000001800081e8     vcruntime:VCRUNTIME140.dll
 0002:000031fc       __IMPORT_DESCRIPTOR_api-ms-win-crt-heap-l1-1-0 00000001800081fc     ucrt:api-ms-win-crt-heap-l1-1-0.dll
 0002:00003210       __IMPORT_DESCRIPTOR_api-ms-win-crt-runtime-l1-1-0 0000000180008210     ucrt:api-ms-win-crt-runtime-l1-1-0.dll
 0002:00003224       __IMPORT_DESCRIPTOR_api-ms-win-crt-convert-l1-1-0 0000000180008224     ucrt:api-ms-win-crt-convert-l1-1-0.dll
 0002:00003238       __IMPORT_DESCRIPTOR_api-ms-win-crt-stdio-l1-1-0 0000000180008238     ucrt:api-ms-win-crt-stdio-l1-1-0.dll
 0002:0000324c       __IMPORT_DESCRIPTOR_api-ms-win-crt-string-l1-1-0 000000018000824c     ucrt:api-ms-win-crt-string-l1-1-0.dll
 0002:00003260       __NULL_IMPORT_DESCRIPTOR   0000000180008260     kernel32:KERNEL32.dll
 0003:00000030       _Init_global_epoch         0000000180009030     MSVCRT:thread_safe_statics.obj
 0003:00000040       __security_cookie          0000000180009040     MSVCRT:gs_cookie.obj
 0003:00000048       __security_cookie_complement 0000000180009048     MSVCRT:gs_cookie.obj
 0003:00000050       __scrt_native_dllmain_reason 0000000180009050     MSVCRT:utility.obj
 0003:00000058       __isa_available            0000000180009058     MSVCRT:cpu_disp.obj
 0003:0000005c       __isa_enabled              000000018000905c     MSVCRT:cpu_disp.obj
 0003:00000060       __memset_fast_string_threshold 0000000180009060     MSVCRT:cpu_disp.obj
 0003:00000068       __memset_nt_threshold      0000000180009068     MSVCRT:cpu_disp.obj
 0003:00000070       __scrt_ucrt_dll_is_in_use  0000000180009070     MSVCRT:ucrt_stubs.obj
 0003:00000080       g_wrongHeapCallbacks       0000000180009080     libobjsize001.obj
 0003:00000100       g_szTagInfo                0000000180009100     libobjsize001.obj
 0003:00002040       g_tagFlags                 000000018000b040     libobjsize001.obj
 0003:00002428       g_refsToVerifyCnt          000000018000b428     libobjsize001.obj
 0003:0000242c       g_fakeUserData             000000018000b42c     libobjsize001.obj
 0003:00002430       g_tagVisitCount            000000018000b430     libobjsize001.obj
 0003:000033d0       g_refsToVerify             000000018000c3d0     libobjsize001.obj
 0003:0001aad0       g_userDataError            0000000180023ad0     libobjsize001.obj
 0003:0001ac70       ?_OptionsStorage@?1??__local_stdio_printf_options@@9@4_KA 0000000180023c70     libobjsize001.obj
 0003:0001b238       _tls_index                 0000000180024238     MSVCRT:tlssup.obj
 0003:0001b240       __scrt_current_native_startup_state 0000000180024240     MSVCRT:utility.obj
 0003:0001b248       __scrt_native_startup_lock 0000000180024248     MSVCRT:utility.obj
 0003:0001b288       __scrt_debugger_hook_flag  0000000180024288     MSVCRT:utility_desktop.obj
 0003:0001b290       ?__type_info_root_node@@3U__type_info_node@@A 0000000180024290     MSVCRT:tncleanup.obj
 0003:0001b2a0       ?_OptionsStorage@?1??__local_stdio_scanf_options@@9@4_KA 00000001800242a0     MSVCRT:default_local_stdio_options.obj
 0003:0001b2a8       __favor                    00000001800242a8     MSVCRT:cpu_disp.obj
 0003:0001b2b0       __dyn_tls_init_callback    00000001800242b0     <common>

 entry point at        0001:00003070

 Static symbols

 0000:fffd9000       .debug$S                   0000000180000000     objsize001.exp
 0000:fffd9000       .debug$S                   0000000180000000     vcruntime:VCRUNTIME140.dll
 0000:fffd9000       .debug$S                   0000000180000000     vcruntime:VCRUNTIME140.dll
 0000:fffd9000       .debug$S                   0000000180000000     vcruntime:VCRUNTIME140.dll
 0000:fffd9000       .debug$S                   0000000180000000     vcruntime:VCRUNTIME140.dll
 0000:fffd9000       .debug$S                   0000000180000000     vcruntime:VCRUNTIME140.dll
 0000:fffd9000       .debug$S                   0000000180000000     vcruntime:VCRUNTIME140.dll
 0000:fffd9000       .debug$S                   0000000180000000     vcruntime:VCRUNTIME140.dll
 0000:fffd9000       .debug$S                   0000000180000000     ucrt:api-ms-win-crt-convert-l1-1-0.dll
 0000:fffd9000       .debug$S                   0000000180000000     ucrt:api-ms-win-crt-heap-l1-1-0.dll
 0000:fffd9000       .debug$S                   0000000180000000     ucrt:api-ms-win-crt-heap-l1-1-0.dll
 0000:fffd9000       .debug$S                   0000000180000000     ucrt:api-ms-win-crt-heap-l1-1-0.dll
 0000:fffd9000       .debug$S                   0000000180000000     ucrt:api-ms-win-crt-heap-l1-1-0.dll
 0000:fffd9000       .debug$S                   0000000180000000     ucrt:api-ms-win-crt-runtime-l1-1-0.dll
 0000:fffd9000       .debug$S                   0000000180000000     ucrt:api-ms-win-crt-runtime-l1-1-0.dll
 0000:fffd9000       .debug$S                   0000000180000000     ucrt:api-ms-win-crt-runtime-l1-1-0.dll
 0000:fffd9000       .debug$S                   0000000180000000     ucrt:api-ms-win-crt-runtime-l1-1-0.dll
 0000:fffd9000       .debug$S                   0000000180000000     ucrt:api-ms-win-crt-runtime-l1-1-0.dll
 0000:fffd9000       .debug$S                   0000000180000000     ucrt:api-ms-win-crt-runtime-l1-1-0.dll
 0000:fffd9000       .debug$S                   0000000180000000     ucrt:api-ms-win-crt-runtime-l1-1-0.dll
 0000:fffd9000       .debug$S                   0000000180000000     ucrt:api-ms-win-crt-runtime-l1-1-0.dll
 0000:fffd9000       .debug$S                   0000000180000000     ucrt:api-ms-win-crt-runtime-l1-1-0.dll
 0000:fffd9000       .debug$S                   0000000180000000     ucrt:api-ms-win-crt-runtime-l1-1-0.dll
 0000:fffd9000       .debug$S                   0000000180000000     ucrt:api-ms-win-crt-runtime-l1-1-0.dll
 0000:fffd9000       .debug$S                   0000000180000000     ucrt:api-ms-win-crt-runtime-l1-1-0.dll
 0000:fffd9000       .debug$S                   0000000180000000     ucrt:api-ms-win-crt-runtime-l1-1-0.dll
 0000:fffd9000       .debug$S                   0000000180000000     ucrt:api-ms-win-crt-runtime-l1-1-0.dll
 0000:fffd9000       .debug$S                   0000000180000000     ucrt:api-ms-win-crt-runtime-l1-1-0.dll
 0000:fffd9000       .debug$S                   0000000180000000     ucrt:api-ms-win-crt-runtime-l1-1-0.dll
 0000:fffd9000       .debug$S                   0000000180000000     ucrt:api-ms-win-crt-stdio-l1-1-0.dll
 0000:fffd9000       .debug$S                   0000000180000000     ucrt:api-ms-win-crt-stdio-l1-1-0.dll
 0000:fffd9000       .debug$S                   0000000180000000     ucrt:api-ms-win-crt-stdio-l1-1-0.dll
 0000:fffd9000       .debug$S                   0000000180000000     ucrt:api-ms-win-crt-stdio-l1-1-0.dll
 0000:fffd9000       .debug$S                   0000000180000000     ucrt:api-ms-win-crt-stdio-l1-1-0.dll
 0000:fffd9000       .debug$S                   0000000180000000     ucrt:api-ms-win-crt-stdio-l1-1-0.dll
 0000:fffd9000       .debug$S                   0000000180000000     ucrt:api-ms-win-crt-stdio-l1-1-0.dll
 0000:fffd9000       .debug$S                   0000000180000000     ucrt:api-ms-win-crt-stdio-l1-1-0.dll
 0000:fffd9000       .debug$S                   0000000180000000     ucrt:api-ms-win-crt-stdio-l1-1-0.dll
 0000:fffd9000       .debug$S                   0000000180000000     ucrt:api-ms-win-crt-stdio-l1-1-0.dll
 0000:fffd9000       .debug$S                   0000000180000000     ucrt:api-ms-win-crt-string-l1-1-0.dll
 0000:fffd9000       .debug$S                   0000000180000000     ucrt:api-ms-win-crt-string-l1-1-0.dll
 0000:fffd9000       .debug$S                   0000000180000000     ucrt:api-ms-win-crt-string-l1-1-0.dll
 0000:fffd9000       .debug$S                   0000000180000000     ucrt:api-ms-win-crt-string-l1-1-0.dll
 0000:fffd9000       .debug$S                   0000000180000000     ucrt:api-ms-win-crt-string-l1-1-0.dll
 0000:fffd9000       .debug$S                   0000000180000000     ucrt:api-ms-win-crt-string-l1-1-0.dll
 0000:fffd9000       .debug$S                   0000000180000000     ucrt:api-ms-win-crt-string-l1-1-0.dll
 0000:fffd9000       .debug$S                   0000000180000000     ucrt:api-ms-win-crt-string-l1-1-0.dll
 0000:fffd9000       .debug$S                   0000000180000000     kernel32:KERNEL32.dll
 0000:fffd9000       .debug$S                   0000000180000000     kernel32:KERNEL32.dll
 0000:fffd9000       .debug$S                   0000000180000000     kernel32:KERNEL32.dll
 0000:fffd9000       .debug$S                   0000000180000000     kernel32:KERNEL32.dll
 0000:fffd9000       .debug$S                   0000000180000000     kernel32:KERNEL32.dll
 0000:fffd9000       .debug$S                   0000000180000000     kernel32:KERNEL32.dll
 0000:fffd9000       .debug$S                   0000000180000000     kernel32:KERNEL32.dll
 0000:fffd9000       .debug$S                   0000000180000000     kernel32:KERNEL32.dll
 0000:fffd9000       .debug$S                   0000000180000000     kernel32:KERNEL32.dll
 0000:fffd9000       .debug$S                   0000000180000000     kernel32:KERNEL32.dll
 0000:fffd9000       .debug$S                   0000000180000000     kernel32:KERNEL32.dll
 0000:fffd9000       .debug$S                   0000000180000000     kernel32:KERNEL32.dll
 0000:fffd9000       .debug$S                   0000000180000000     kernel32:KERNEL32.dll
 0000:fffd9000       .debug$S                   0000000180000000     kernel32:KERNEL32.dll
 0000:fffd9000       .debug$S                   0000000180000000     kernel32:KERNEL32.dll
 0000:fffd9000       .debug$S                   0000000180000000     kernel32:KERNEL32.dll
 0000:fffd9000       .debug$S                   0000000180000000     kernel32:KERNEL32.dll
 0000:fffd9000       .debug$S                   0000000180000000     kernel32:KERNEL32.dll
 0000:fffd9000       .debug$S                   0000000180000000     kernel32:KERNEL32.dll
 0000:fffd9000       .debug$S                   0000000180000000     kernel32:KERNEL32.dll
 0000:fffd9000       .debug$S                   0000000180000000     kernel32:KERNEL32.dll
 0000:fffd9000       .debug$S                   0000000180000000     kernel32:KERNEL32.dll
 0000:fffd9000       .debug$S                   0000000180000000     kernel32:KERNEL32.dll
 0000:fffd9000       .debug$S                   0000000180000000     kernel32:KERNEL32.dll
 0000:fffd9000       .debug$S                   0000000180000000     kernel32:KERNEL32.dll
 0000:fffd9000       .debug$S                   0000000180000000     kernel32:KERNEL32.dll
 0000:fffd9000       .debug$S                   0000000180000000     kernel32:KERNEL32.dll
 0000:fffd9000       .debug$S                   0000000180000000     kernel32:KERNEL32.dll
 0001:00000dd4       addRefToVerify             0000000180001dd4 f   libobjsize001.obj
 0001:00000e40       agentProc                  0000000180001e40 f   libobjsize001.obj
 0001:000015d8       agentThreadWrapper         00000001800025d8 f   libobjsize001.obj
 0001:00001744       check_option               0000000180002744 f   libobjsize001.obj
 0001:0000198c       file_basename              000000018000298c f   libobjsize001.obj
 0001:00002550       startAgentThreadWrapper    0000000180003550 f   libobjsize001.obj
 0001:00002890       syncDebuggeeStatus         0000000180003890 f   libobjsize001.obj
 0001:00002b30       capture_previous_context   0000000180003b30 f   MSVCRT:gs_report.obj
 0001:00002ba4       ?__scrt_initialize_thread_safe_statics@@YAHXZ 0000000180003ba4 f   MSVCRT:thread_safe_statics.obj
 0001:00002c74       ?__scrt_uninitialize_thread_safe_statics@@YAXXZ 0000000180003c74 f   MSVCRT:thread_safe_statics.obj
 0001:00002d20       $$000000                   0000000180003d20     MSVCRT:amdsecgs.obj
 0001:00002d50       ?dllmain_crt_dispatch@@YAHQEAUHINSTANCE__@@KQEAX@Z 0000000180003d50 f   MSVCRT:dll_dllmain.obj
 0001:00002da0       ?dllmain_crt_process_attach@@YAHQEAUHINSTANCE__@@QEAX@Z 0000000180003da0 f   MSVCRT:dll_dllmain.obj
 0001:00002eb8       ?dllmain_crt_process_detach@@YAH_N@Z 0000000180003eb8 f   MSVCRT:dll_dllmain.obj
 0001:00002f3c       ?dllmain_dispatch@@YAHQEAUHINSTANCE__@@KQEAX@Z 0000000180003f3c f   MSVCRT:dll_dllmain.obj
 0001:00003950       $$000000                   0000000180004950     MSVCRT:guard_dispatch.obj
 0001:00003970       $$000000                   0000000180004970     MSVCRT:guard_xfg_dispatch.obj
 0001:00003986       ?fin$0@?0??dllmain_crt_process_attach@@YAHQEAUHINSTANCE__@@QEAX@Z@4HA 0000000180004986 f   MSVCRT:dll_dllmain.obj
 0001:0000399d       ?fin$0@?0??dllmain_crt_process_detach@@YAH_N@Z@4HA 000000018000499d f   MSVCRT:dll_dllmain.obj
 0001:000039b6       ?fin$1@?0??dllmain_crt_process_detach@@YAH_N@Z@4HA 00000001800049b6 f   MSVCRT:dll_dllmain.obj
 0001:000039ca       ?filt$0@?0??dllmain_dispatch@@YAHQEAUHINSTANCE__@@KQEAX@Z@4HA 00000001800049ca f   MSVCRT:dll_dllmain.obj
 0001:00003a00       __scrt_is_nonwritable_in_current_image$filt$0 0000000180004a00 f   MSVCRT:utility.obj
 0002:00000218       ?__scrt_initialize_tss_var@@3P6AHXZEA 0000000180005218     MSVCRT:thread_safe_statics.obj
 0002:00000340       ?opcLengths@@3QBEB         0000000180005340     libobjsize001.obj
 0002:00002470       GS_ExceptionPointers       0000000180007470     MSVCRT:gs_report.obj
 0002:00002b30       $unwind$fprintf            0000000180007b30     libobjsize001.obj
 0002:00002b3c       $unwind$printf             0000000180007b3c     libobjsize001.obj
 0002:00002b48       $unwind$?NewObject@JNIEnv_@@QEAAPEAV_jobject@@PEAV_jclass@@PEAU_jmethodID@@ZZ 0000000180007b48     libobjsize001.obj
 0002:00002b48       $unwind$nsk_lcomplain      0000000180007b48     libobjsize001.obj
 0002:00002b48       $unwind$nsk_ldisplay       0000000180007b48     libobjsize001.obj
 0002:00002b50       $unwind$nsk_jvmti_waitForSync 0000000180007b50     libobjsize001.obj
 0002:00002b50       $unwind$nsk_lvdisplay      0000000180007b50     libobjsize001.obj
 0002:00002b50       $unwind$_RTC_Initialize    0000000180007b50     MSVCRT:initsect.obj
 0002:00002b50       $unwind$_RTC_Terminate     0000000180007b50     MSVCRT:initsect.obj
 0002:00002b50       $unwind$?__scrt_initialize_thread_safe_statics@@YAHXZ 0000000180007b50     MSVCRT:thread_safe_statics.obj
 0002:00002b5c       $unwind$nsk_complain       0000000180007b5c     libobjsize001.obj
 0002:00002b5c       $unwind$nsk_printf         0000000180007b5c     libobjsize001.obj
 0002:00002b64       $unwind$nsk_lvcomplain     0000000180007b64     libobjsize001.obj
 0002:00002b7c       $unwind$nsk_ltrace         0000000180007b7c     libobjsize001.obj
 0002:00002b7c       $unwind$__report_gsfailure 0000000180007b7c     MSVCRT:gs_report.obj
 0002:00002b84       $unwind$nsk_lvtrace        0000000180007b84     libobjsize001.obj
 0002:00002b84       $unwind$__raise_securityfailure 0000000180007b84     MSVCRT:gs_report.obj
 0002:00002b84       $unwind$__scrt_initialize_crt 0000000180007b84     MSVCRT:utility.obj
 0002:00002b84       $unwind$__scrt_initialize_onexit_tables 0000000180007b84     MSVCRT:utility.obj
 0002:00002b84       $unwind$__scrt_release_startup_lock 0000000180007b84     MSVCRT:utility.obj
 0002:00002b84       $unwind$__scrt_uninitialize_crt 0000000180007b84     MSVCRT:utility.obj
 0002:00002b84       $unwind$_onexit            0000000180007b84     MSVCRT:utility.obj
 0002:00002b8c       $unwind$nsk_lverify        0000000180007b8c     libobjsize001.obj
 0002:00002b9c       $unwind$nsk_vprintf        0000000180007b9c     libobjsize001.obj
 0002:00002bac       $unwind$?nsk_jni_lverify@@YAHHPEAUJNIEnv_@@HQEBDH1ZZ 0000000180007bac     libobjsize001.obj
 0002:00002bc0       $unwind$?nsk_jni_check_exception@@YAHPEAUJNIEnv_@@QEBDH@Z 0000000180007bc0     libobjsize001.obj
 0002:00002bdc       $unwind$nsk_jvmti_parseOptions 0000000180007bdc     libobjsize001.obj
 0002:00002bf8       $unwind$nsk_jvmti_createJVMTIEnv 0000000180007bf8     libobjsize001.obj
 0002:00002c0c       $unwind$Java_nsk_jvmti_unit_FollowReferences_FollowRefObjects_resetTags 0000000180007c0c     libobjsize001.obj
 0002:00002c0c       $unwind$addRefToVerify     0000000180007c0c     libobjsize001.obj
 0002:00002c0c       $unwind$nsk_jvmti_resetAgentData 0000000180007c0c     libobjsize001.obj
 0002:00002c0c       $unwind$nsk_jvmti_resumeSync 0000000180007c0c     libobjsize001.obj
 0002:00002c0c       $unwind$nsk_jvmti_setFailStatus 0000000180007c0c     libobjsize001.obj
 0002:00002c0c       $unwind$__scrt_initialize_default_local_stdio_options 0000000180007c0c     MSVCRT:default_local_stdio_options.obj
 0002:00002c0c       $unwind$?dllmain_crt_dispatch@@YAHQEAUHINSTANCE__@@KQEAX@Z 0000000180007c0c     MSVCRT:dll_dllmain.obj
 0002:00002c0c       $unwind$DllMain            0000000180007c0c     MSVCRT:dll_dllmain_stub.obj
 0002:00002c0c       $unwind$__GSHandlerCheck   0000000180007c0c     MSVCRT:gshandler.obj
 0002:00002c0c       $unwind$?__scrt_uninitialize_thread_safe_statics@@YAXXZ 0000000180007c0c     MSVCRT:thread_safe_statics.obj
 0002:00002c0c       $unwind$__scrt_acquire_startup_lock 0000000180007c0c     MSVCRT:utility.obj
 0002:00002c0c       $unwind$__scrt_dllmain_after_initialize_c 0000000180007c0c     MSVCRT:utility.obj
 0002:00002c0c       $unwind$__scrt_dllmain_before_initialize_c 0000000180007c0c     MSVCRT:utility.obj
 0002:00002c0c       $unwind$__scrt_dllmain_crt_thread_attach 0000000180007c0c     MSVCRT:utility.obj
 0002:00002c0c       $unwind$__scrt_dllmain_crt_thread_detach 0000000180007c0c     MSVCRT:utility.obj
 0002:00002c0c       $unwind$__scrt_dllmain_uninitialize_c 0000000180007c0c     MSVCRT:utility.obj
 0002:00002c0c       $unwind$__scrt_dllmain_uninitialize_critical 0000000180007c0c     MSVCRT:utility.obj
 0002:00002c0c       $unwind$atexit             0000000180007c0c     MSVCRT:utility.obj
 0002:00002c14       $unwind$nsk_jvmti_lverify  0000000180007c14     libobjsize001.obj
 0002:00002c28       $unwind$exitOnError        0000000180007c28     libobjsize001.obj
 0002:00002c38       $unwind$check_option       0000000180007c38     libobjsize001.obj
 0002:00002c38       $unwind$_DllMainCRTStartup 0000000180007c38     MSVCRT:dll_dllmain.obj
 0002:00002c48       $unwind$Java_nsk_share_jvmti_ArgumentHandler_getAgentOptionsString 0000000180007c48     libobjsize001.obj
 0002:00002c5c       $unwind$Java_nsk_jvmti_unit_FollowReferences_FollowRefObjects_getTag 0000000180007c5c     libobjsize001.obj
 0002:00002c5c       $unwind$Java_nsk_share_jvmti_DebugeeClass_checkStatus 0000000180007c5c     libobjsize001.obj
 0002:00002c5c       $unwind$agentThreadWrapper 0000000180007c5c     libobjsize001.obj
 0002:00002c6c       $unwind$startAgentThreadWrapper 0000000180007c6c     libobjsize001.obj
 0002:00002c88       $unwind$syncDebuggeeStatus 0000000180007c88     libobjsize001.obj
 0002:00002c88       $unwind$__scrt_dllmain_exception_filter 0000000180007c88     MSVCRT:utility.obj
 0002:00002c9c       $unwind$Java_nsk_share_jvmti_DebugeeClass_resetAgentData 0000000180007c9c     libobjsize001.obj
 0002:00002ca4       $unwind$MA_checkStatus     0000000180007ca4     libobjsize001.obj
 0002:00002cb8       $unwind$Java_nsk_jvmti_unit_FollowReferences_FollowRefObjects_setTag 0000000180007cb8     libobjsize001.obj
 0002:00002cd0       $unwind$Java_nsk_jvmti_unit_FollowReferences_FollowRefObjects_addRefToVerify 0000000180007cd0     libobjsize001.obj
 0002:00002cec       $unwind$Agent_Initialize   0000000180007cec     libobjsize001.obj
 0002:00002d08       $unwind$agentProc          0000000180007d08     libobjsize001.obj
 0002:00002d24       $unwind$capture_previous_context 0000000180007d24     MSVCRT:gs_report.obj
 0002:00002d30       $unwind$__GSHandlerCheckCommon 0000000180007d30     MSVCRT:gshandler.obj
 0002:00002d38       $xdatasym                  0000000180007d38     MSVCRT:amdsecgs.obj
 0002:00002d3c       $unwind$?dllmain_crt_process_attach@@YAHQEAUHINSTANCE__@@QEAX@Z 0000000180007d3c     MSVCRT:dll_dllmain.obj
 0002:00002d78       $unwind$?fin$0@?0??dllmain_crt_process_attach@@YAHQEAUHINSTANCE__@@QEAX@Z@4HA 0000000180007d78     MSVCRT:dll_dllmain.obj
 0002:00002d78       $unwind$?fin$0@?0??dllmain_crt_process_detach@@YAH_N@Z@4HA 0000000180007d78     MSVCRT:dll_dllmain.obj
 0002:00002d78       $unwind$?fin$1@?0??dllmain_crt_process_detach@@YAH_N@Z@4HA 0000000180007d78     MSVCRT:dll_dllmain.obj
 0002:00002d80       $unwind$?dllmain_crt_process_detach@@YAH_N@Z 0000000180007d80     MSVCRT:dll_dllmain.obj
 0002:00002dd4       $unwind$?dllmain_dispatch@@YAHQEAUHINSTANCE__@@KQEAX@Z 0000000180007dd4     MSVCRT:dll_dllmain.obj
 0002:00002dfc       $unwind$?filt$0@?0??dllmain_dispatch@@YAHQEAUHINSTANCE__@@KQEAX@Z@4HA 0000000180007dfc     MSVCRT:dll_dllmain.obj
 0002:00002e04       $unwind$__scrt_is_nonwritable_in_current_image 0000000180007e04     MSVCRT:utility.obj
 0002:00002e24       $unwind$__scrt_is_nonwritable_in_current_image$filt$0 0000000180007e24     MSVCRT:utility.obj
 0002:00002e2c       $unwind$__scrt_fastfail    0000000180007e2c     MSVCRT:utility_desktop.obj
 0002:00002e3c       $unwind$__security_init_cookie 0000000180007e3c     MSVCRT:gs_support.obj
 0002:00002e48       $unwind$__isa_available_init 0000000180007e48     MSVCRT:cpu_disp.obj
 0002:00002e58       $xdatasym                  0000000180007e58     MSVCRT:guard_dispatch.obj
 0002:00002e60       $xdatasym                  0000000180007e60     MSVCRT:guard_xfg_dispatch.obj
 0002:00002e70       .edata                     0000000180007e70     objsize001.exp
 0002:00002e98       rgpv                       0000000180007e98     objsize001.exp
 0002:00002ed0       rgszName                   0000000180007ed0     objsize001.exp
 0002:00002f08       rgwOrd                     0000000180007f08     objsize001.exp
 0002:00002f24       szName                     0000000180007f24     objsize001.exp
 0002:00002f33       $N00001                    0000000180007f33     objsize001.exp
 0002:00002f42       $N00002                    0000000180007f42     objsize001.exp
 0002:00002f4f       $N00003                    0000000180007f4f     objsize001.exp
 0002:00002f94       $N00004                    0000000180007f94     objsize001.exp
 0002:00002fd1       $N00005                    0000000180007fd1     objsize001.exp
 0002:00003019       $N00006                    0000000180008019     objsize001.exp
 0002:00003059       $N00007                    0000000180008059     objsize001.exp
 0002:00003096       $N00008                    0000000180008096     objsize001.exp
 0002:000030d1       $N00009                    00000001800080d1     objsize001.exp
 0002:000030ff       $N00010                    00000001800080ff     objsize001.exp
 0002:00003130       $N00011                    0000000180008130     objsize001.exp
 0002:0000315f       $N00012                    000000018000815f     objsize001.exp
 0002:0000318e       $N00013                    000000018000818e     objsize001.exp
 0002:000031c3       $N00014                    00000001800081c3     objsize001.exp
 0002:0000362a       .idata$6                   000000018000862a     kernel32:KERNEL32.dll
 0002:0000368e       .idata$6                   000000018000868e     vcruntime:VCRUNTIME140.dll
 0002:00003820       .idata$6                   0000000180008820     ucrt:api-ms-win-crt-heap-l1-1-0.dll
 0002:00003840       .idata$6                   0000000180008840     ucrt:api-ms-win-crt-runtime-l1-1-0.dll
 0002:00003862       .idata$6                   0000000180008862     ucrt:api-ms-win-crt-convert-l1-1-0.dll
 0002:00003884       .idata$6                   0000000180008884     ucrt:api-ms-win-crt-stdio-l1-1-0.dll
 0002:000038a4       .idata$6                   00000001800088a4     ucrt:api-ms-win-crt-string-l1-1-0.dll
 0003:00000000       ?codeAttributeName@@3PEBDEB 0000000180009000     libobjsize001.obj
 0003:00000008       ?lineNumberAttributeName@@3PEBDEB 0000000180009008     libobjsize001.obj
 0003:00000010       ?localVarAttributeName@@3PEBDEB 0000000180009010     libobjsize001.obj
 0003:00000018       ?localVarTypeAttributeName@@3PEBDEB 0000000180009018     libobjsize001.obj
 0003:00000020       ?stackMapAttributeName@@3PEBDEB 0000000180009020     libobjsize001.obj
 0003:00000028       ?callBytes@@3PAEA          0000000180009028     libobjsize001.obj
 0003:0000002c       ?allocBytes@@3PAEA         000000018000902c     libobjsize001.obj
 0003:0001aad4       redefineAttempted          0000000180023ad4     libobjsize001.obj
 0003:0001aad8       nsk_context                0000000180023ad8     libobjsize001.obj
 0003:0001aae4       redefineSucceed            0000000180023ae4     libobjsize001.obj
 0003:0001aae8       agentFailed                0000000180023ae8     libobjsize001.obj
 0003:0001aaec       currentAgentStatus         0000000180023aec     libobjsize001.obj
 0003:0001aaf0       context                    0000000180023af0     libobjsize001.obj
 0003:0001aba8       agentThread                0000000180023ba8     libobjsize001.obj
 0003:0001abb0       agentThreadProc            0000000180023bb0     libobjsize001.obj
 0003:0001abb8       agentThreadArg             0000000180023bb8     libobjsize001.obj
 0003:0001abc0       agent_data                 0000000180023bc0     libobjsize001.obj
 0003:0001abd0       jvmti_env                  0000000180023bd0     libobjsize001.obj
 0003:0001abd8       jvm                        0000000180023bd8     libobjsize001.obj
 0003:0001abe0       jni_env                    0000000180023be0     libobjsize001.obj
 0003:0001abe8       checkStatus_func           0000000180023be8     libobjsize001.obj
 0003:0001abf0       ?codeAttributeIndex@@3GA   0000000180023bf0     libobjsize001.obj
 0003:0001abf4       ?lineNumberAttributeIndex@@3GA 0000000180023bf4     libobjsize001.obj
 0003:0001abf8       ?localVarAttributeIndex@@3GA 0000000180023bf8     libobjsize001.obj
 0003:0001abfc       ?localVarTypeAttributeIndex@@3GA 0000000180023bfc     libobjsize001.obj
 0003:0001ac00       ?stackMapAttributeIndex@@3GA 0000000180023c00     libobjsize001.obj
 0003:0001ac04       ?stackFrameOffset@@3GA     0000000180023c04     libobjsize001.obj
 0003:0001ac08       ?mode@@3HA                 0000000180023c08     libobjsize001.obj
 0003:0001ac0c       ?constantPoolSize@@3GA     0000000180023c0c     libobjsize001.obj
 0003:0001ac10       ?orig@@3PEBEEB             0000000180023c10     libobjsize001.obj
 0003:0001ac18       ?gen@@3PEAEEA              0000000180023c18     libobjsize001.obj
 0003:0001ac20       ?inputPos@@3PEAEEA         0000000180023c20     libobjsize001.obj
 0003:0001ac28       ?endPos@@3PEBEEB           0000000180023c28     libobjsize001.obj
 0003:0001ac30       ?genPos@@3PEAEEA           0000000180023c30     libobjsize001.obj
 0003:0001ac38       ?markPos@@3PEAEEA          0000000180023c38     libobjsize001.obj
 0003:0001ac40       ?constantPool@@3PEAPEADEA  0000000180023c40     libobjsize001.obj
 0003:0001ac48       ?constantPoolCount@@3GA    0000000180023c48     libobjsize001.obj
 0003:0001ac4c       ?zeroBytes@@3PAEA          0000000180023c4c     libobjsize001.obj
 0003:0001ac50       ?codeLength@@3IA           0000000180023c50     libobjsize001.obj
 0003:0001ac58       ?map@@3PEAIEA              0000000180023c58     libobjsize001.obj
 0003:0001ac60       ?widening@@3PEACEA         0000000180023c60     libobjsize001.obj
 0003:0001ac68       timeout                    0000000180023c68     libobjsize001.obj
 0003:0001ac80       GS_ExceptionRecord         0000000180023c80     MSVCRT:gs_report.obj
 0003:0001ad20       GS_ContextRecord           0000000180023d20     MSVCRT:gs_report.obj
 0003:0001b1f0       ?g_tss_cv@@3U_RTL_CONDITION_VARIABLE@@A 00000001800241f0     MSVCRT:thread_safe_statics.obj
 0003:0001b1f8       ?g_tss_event@@3PEAXEA      00000001800241f8     MSVCRT:thread_safe_statics.obj
 0003:0001b200       ?g_tss_mutex@@3U_RTL_CRITICAL_SECTION@@A 0000000180024200     MSVCRT:thread_safe_statics.obj
 0003:0001b228       ?g_sleep_condition_variable_cs@@3P6AHPEAU_RTL_CONDITION_VARIABLE@@PEAU_RTL_CRITICAL_SECTION@@K@ZEA 0000000180024228     MSVCRT:thread_safe_statics.obj
 0003:0001b230       ?g_wake_all_condition_variable@@3P6AXPEAU_RTL_CONDITION_VARIABLE@@@ZEA 0000000180024230     MSVCRT:thread_safe_statics.obj
 0003:0001b23c       ?__proc_attached@@3HA      000000018002423c     MSVCRT:dll_dllmain.obj
 0003:0001b250       ?is_initialized_as_dll@@3_NA 0000000180024250     MSVCRT:utility.obj
 0003:0001b251       ?module_local_atexit_table_initialized@@3_NA 0000000180024251     MSVCRT:utility.obj
 0003:0001b258       ?module_local_atexit_table@@3U_onexit_table_t@@A 0000000180024258     MSVCRT:utility.obj
 0003:0001b270       ?module_local_at_quick_exit_table@@3U_onexit_table_t@@A 0000000180024270     MSVCRT:utility.obj
